:020000000E00F0
:08001000000C2500FF0C260086
:08001800FF0C27005E000F0C35
:0800200005000F0C0600000CA6
:0800280007005F00000C050059
:08003000F00C0600FF0C0700B4
:080038007F0C020006052605FD
:080040006C00250AEB02280AFE
:080048006C021E0C2B000206E5
:08005000290AA607330A8607FE
:08005800300A2E0A1100000A13
:0800600000001200000A340A3E
:040068001300000A77
:08040000030C2900000C2A0086
:08040800280A06054F0C28002C
:08041000E802080A0B0A0502CC
:08041800080E000D2500FA0C8E
:080420002800E802110AFA0CA1
:080428002800E802150A950CFA
:080430002800E802190A1C0A69
:08043800E902220A2A02430630
:08044000330A0206250AEA0056
:080448000207260A0000280A41
:0804500006020104210426004C
:080458003A0C2800E8022E0A0C
:0804600000000000050A170C62
:080468002900000C2A005B0AC8
:0804700006054F0C2800E8020C
:080478003B0A3E0A0502080ED2
:08048000000D2500FA0C280014
:08048800E802440AFA0C280006
:08049000E802480A950C28005F
:08049800E8024C0A4F0AE902D8
:0804A000550A2A024306660A10
:0804A8000207580AEA000206EF
:0804B000590A00005B0A060274
:0804B8000104210526003A0CA5
:0804C0002800E802610A0000B7
:0804C8000000380AE00C2900D5
:0804D000000C2A00CE0A06050B
:0804D8004F0C2800E8026E0A37
:0804E000710A0502080E070D68
:0804E80025004B0C2800E8027E
:0804F000770A7A0A0502080EE2
:0804F800060D25004B0C280045
:08050000E802800A830A0502EB
:08050800080E050D25004B0C47
:080510002800E802890A8C0AA8
:080518000502080E040D250088
:080520004B0C2800E802920ACE
:08052800950A0502080E030DFF
:0805300025004B0C2800E80235
:080538009B0A9E0A0502080E51
:08054000020D25004B0C280000
:08054800E802A40AA70A05025B
:08055000080E010D25004B0C03
:080558002800E802AD0AB00A18
:080560000502080E000D250044
:080568004B0C2800E802B60A62
:08057000B90A0502080E000D96
:080578002500230C2800E80215
:08058000BF0AC20AE902C80A21
:080588002A024306D70A02060D
:08059000CB0AEA000207CC0AC5
:080598000000CE0ACF0A0604A0
:0805A0003A0C2800E802D20A1F
:0805A800000000006B0A0D0CBD
:0805B0002900000C2A00000BD9
:0805B80006054F0C2800E802C3
:0805C000DF0AE20A0502080E41
:0805C800000D2500FA0C2800CB
:0805D000E802E80AFA0C280019
:0805D800E802EC0A900C280077
:0805E000E802F00AF30AE90247
:0805E800FA0A2A024307FB0A8C
:0805F0001000220AFD0AEA00D6
:0805F8000207FE0A0000000BDF
:08060000050C2800E802020BC2
:08060800050B06043A0C280062
:08061000E802080B00000000E5
:02061800DC0AFA
:08080000040C2900000C2A0081
:08080800240A0605360C280045
:08081000E802080A00000000E4
:080818000502080E000D250089
:08082000FA0C2800E802120A9C
:08082800A50C2800E802160AE5
:08083000E9021E0A2A02430638
:080838002F0A0206210AEA0062
:080840000207220A0000240A4D
:08084800060201042104260050
:08085000240C2800E8022A0A2A
:0808580000000000050A190C64
:080860002900000C2A00530AD4
:080868000605360C2800E80229
:08087000370A00000000050238
:08087800080E000D2500FA0C2A
:080880002800E802410AA50C62
:080888002800E802450AE9021C
:080890004D0A2A0243065E0A2C
:080898000207500AEA00020603
:0808A000510A0000530A060290
:0808A800010421052600240CC7
:0808B0002800E802590A0000CB
:0808B8000000340A800C290045
:0808C000010C2A00BE0A060526
:0808C800360C2800E802660A64
:0808D000000000000502080E03
:0808D800070D25002F0C28007C
:0808E000E802700A0502080E8F
:0808E800060D25002F0C28006D
:0808F000E802780A0502080E77
:0808F800050D25002F0C28005E
:08090000E802800A0502080E5E
:08090800040D25002F0C28004E
:08091000E802880A0502080E46
:08091800030D25002F0C28003F
:08092000E802900A0502080E2E
:08092800020D25002F0C280030
:08093000E802980A0502080E16
:08093800010D25002F0C280021
:08094000E802A00A0502080EFE
:08094800000D25002F0C280012
:08095000E802A80A0502080EE6
:08095800000D25001F0C280012
:08096000E802B00AE902B80A3E
:080968002A024306C70A020639
:08097000BB0AEA000207BC0A01
:080978000000BE0ABF0A0604DC
:08098000240C2800E802C20A61
:0809880000000000630A0B0CE3
:080990002900000C2A00EC0A0A
:080998000605360C2800E802F8
:0809A000CF0A0000000005026F
:0809A800080E000D2500FA0CF9
:0809B0002800E802D90AA00C9E
:0809B8002800E802DD0AE90253
:0809C000E60A2A024307E70AD8
:0809C8001000220AE90AEA000E
:0809D0000207EA0A0000EC0A2C
:0809D800050C2800E802EE0AFC
:0809E000F10A0604240C2800B2
:0809E800E802F40A000000001F
:0209F000CC0A2F
:080C0000030C2900000C2A007E
:080C0800240A0605270C280050
:080C1000E802080A00000502D9
:080C1800080E000D2500FA0C86
:080C20002800E802110A3D0C56
:080C28002800E802150A180A71
:080C3000E9021E0A2A02430634
:080C38002D0A0206210AEA0060
:080C40000207220A0000240A49
:080C480006020104210426004C
:080C5000250C2800E8022A0A25
:080C5800050A210C2900000C23
:080C60002A00510A0605270CC9
:080C68002800E802350A000033
:080C70000502080E000D25002D
:080C7800FA0C2800E8023E0A14
:080C80003D0C2800E802420AC5
:080C8800450AE9024B0A2A02A9
:080C900043065A0A02074E0A4E
:080C9800EA0002064F0A000009
:080CA000510A060201042105BE
:080CA8002600250C2800E802DB
:080CB000570A320AE00C29008A
:080CB800010C2A00BA0A06052E
:080CC000270C2800E802620A7B
:080CC80000000502080E070DF3
:080CD0002500240C2800E802B5
:080CD8006B0A0502080E060D6F
:080CE0002500240C2800E802A5
:080CE800730A0502080E050D58
:080CF0002500240C2800E80295
:080CF8007B0A0502080E040D41
:080D00002500240C2800E80284
:080D0800830A0502080E030D29
:080D10002500240C2800E80274
:080D18008B0A0502080E020D12
:080D20002500240C2800E80264
:080D2800930A0502080E010DFB
:080D30002500240C2800E80254
:080D38009B0A0502080E000DE4
:080D40002500240C2800E80244
:080D4800A30A0502080E000DCC
:080D500025000F0C2800E80249
:080D5800AB0AAE0AE902B40A7D
:080D60002A024306C10A020643
:080D6800B70AEA000207B80A0D
:080D70000000BA0ABB0A0604E8
:080D7800250C2800E802BE0A68
:080D80005F0A0E0C2900000CB3
:080D88002A00E60A0605270C0B
:080D90002800E802C90A000076
:080D98000502080E000D250004
:080DA000FA0C2800E802D20A57
:080DA800380C2800E802D60A0D
:080DB000D90AE902E00A2A0257
:080DB8004307E10A1000220AC2
:080DC000E30AEA000207E40A5D
:080DC8000000E60A050C2800FA
:080DD000E802E80AEB0A060440
:080DD800250C2800E802EE0AD8
:020DE000C60A41
:020FFE00080ADF
:08200000F50FF00FF40FF10FD2
:08200800F50FF40FF40FF70FC0
:08201000F40FF50FF40FFE0FB1
:08201800FF0FFF0FFF0FFF0F88
:10202000FA033F0FFFFF02ABFA0280F00000FFFF50
:00000001FF
